S02000006F70656E626C745F6F6C696D65785F65666D3332673838302E7372656320
S1130000780200206D1C0000911C0000911C00006F
S1130010911C0000911C0000911C0000911C000028
S1130020911C0000911C0000911C0000911C000018
S1130030911C0000911C0000911C0000911C000008
S1130040911C0000911C0000911C0000911C0000F8
S1130050911C0000911C0000911C0000911C0000E8
S1130060911C0000911C0000911C0000911C0000D8
S1130070911C0000911C0000911C0000911C0000C8
S1130080911C0000911C0000911C0000911C0000B8
S1130090911C0000911C0000911C0000911C0000A8
S11300A0911C0000911C0000911C0000911C000098
S10B00B0911C0000911C0000EA
S11300B8890011EB401010F1844002607047DFF8AA
S11300C88405006810F007010029012903D9891E55
S11300D8012904D906E0012161F3020002E00321A9
S11300E861F30200DFF85C1508607047B0FA80F02D
S11300F8D0F11F007047DFF84C150968DFF8482570
S1130108821ADFF848359A420BD211F00702921E80
S1130118012A03D8032262F3020102E0012262F3F6
S11301280201DFF8242590420AD211F00700801E4C
S1130138012803D8022060F3020101E0C908C900BC
S1130148DFF8000501607047DFF80405704780B5E3
S1130158DFF8000500F09DF9C0B2072804D008288C
S113016805D100F0AEFA03E0FFF7EEFF00E000204F
S113017802BD80B5DFF8E0140968C0B24000C14090
S113018811F0030000280FD0022806D002D3032858
S113019806D00BE000F0CFFA09E000F0CFFA06E051
S11301A800F084FA400802E0002000E0002002BDCC
S11301B8DFF8A8140968C90704D4DFF8A414096887
S11301C80142FAD1704710B50C00C0F3031101299C
S11301D807D0C0F09A80032925D010D3042967D00A
S11301E893E02000FFF782FF0400DFF88004006832
S11301F8000900012043DFF87414086085E0FFF764
S11302085EFF2000FFF772FF0400DFF86404006853
S1130218000900012043DFF85814086000F046FA8A
S1130228FFF769FF71E0DFF84C14884208D0DFF863
S11302384814884215D0DFF84814884223D036E0A1
S11302480420FFF7B5FF2000FFF750FF0400DFF894
S11302582C040068000900012043DFF8201408601A
S113026825E00420FFF7A4FF2000FFF73FFF040068
S1130278DFF80804006830F0F00050EA0410DFF8F2
S1130288FC13086013E00420FFF792FF2000FFF737
S11302982DFF0400DFF8E403006830F44070B4F183
S11302A8100150EA0120DFF8D4130860FFE72CE0BE
S11302B8DFF8D013884204D0DFF8CC13884211D079
S11302C822E04020FFF774FF2000FFF70FFF04002F
S11302D8DFF8B8030068800880002043DFF8AC1317
S11302E8086011E04020FFF763FF2000FFF7FEFEDF
S11302F80400DFF89803006830F0300050EA041076
S1130308DFF888130860FFE7FFE710BD70B50C003D
S11303180021C0F30322D2B2012A09D029D3032A27
S113032819D015D3052A1DD018D3062A1ED020E0CB
S1130338DFF83853C0F30436002902D00800FFF769
S113034837FFE4B2220031002800FFF7B1FE70BD88
S1130358DFF83C53EEE7DFF83C53EBE7DFF83853BC
S11303680121E7E7DFF834531021E3E7DFF83053DE
S1130378E0E7ECE780B510F47810002824D0B0F555
S1130388003F24D0B0F5802F2AD0B0F5C02F2AD052
S1130398B0F5002F2BD0B0F5202F32D0B0F5402F78
S11303A839D0B0F5602F41D0B0F5901F51D0B0F5D9
S11303B8A01F52D0B0F5B01F59D0B0F5C01F60D0FF
S11303C8B0F5D01F60D062E000F07BF960E000F087
S11303D878F9DFF89812096811F00F01C84057E05E
S11303E800F064F954E00020FFF7C3FE50E0002059
S11303F8FFF7BFFEDFF88412096811F00F01C84047
S113040846E00020FFF7B5FEDFF870120968C1F373
S11304180311C8403CE00020FFF7ABFEDFF85C1294
S11304280968090A11F00301C84031E00020FFF708
S1130438A0FEDFF848120968090A11F00301C84050
S1130448DFF86012096811F00701491CB0FBF1F0EC
S11304581EE00120FFF78DFE1AE00120FFF789FE58
S1130468DFF82812096811F00301C84010E00120E0
S1130478FFF77FFEDFF814120968C1F30111C840C1
S113048806E0FFF764FE03E0FFF75EFE00E00020ED
S113049802BD012110F00F00012806D036D303282D
S11304A82DD018D304282FD030E0DFF8BC01006821
S11304B810F47050B0F5006F09D0B0F5805F04D027
S11304C8B0F5005F05D1022104E0032102E0042114
S11304D800E005211BE0DFF88001006810F003004C
S11304E8012804D009D3032805D002D305E0032149
S11304F804E0022102E0062100E0012107E0DFF820
S113050858010068012102E0072100E000210800E9
S1130518C0B2704710B50324032310F00F00020083
S1130528521E03D0521E012A27D956E0C9B2022905
S113053806D021D3042919D015D3052919D01BE0D5
S113054804240023012201211800C0B200F046F857
S1130558FFF7B5FD4348046000F00CF900F0A6F875
S1130568FFF7C9FD39E003240123EBE70224022342
S1130578E8E701240323E5E72FE0022801D100245A
S113058800E00224C9B2012906D002290FD00329A8
S113059814D0062919D01FE000202F490968032226
S11305A8A2409143A04008432B49086015E001226A
S11305B80121002000F012F80220EEE701220121B7
S11305C8012000F00BF80120E7E70122022131485D
S11305D8FFF76EFD0320E0E7FFE710BD10B5C0B2DA
S11305E8002821D0022813D01AD3042814D022D2E8
S11305F8012302240220C9B200291DD02A490B6014
S1130608D2B2002A1AD018490968014216D1FAE769
S1130618042308240820EEE7102320242020EAE7F6
S1130628402380248020E6E74FF480734FF400745D
S11306384FF40070DFE703E01B48046000F09AF809
S113064810BD000004000C400124F4000024F40050
S1130658809FD5000400180028800C4054800C406A
S113066850800C4024800C402C800C4008800C40A6
S113067804800C403004080030140A0068800C40E0
S113068830000C00400514004015160070800C4022
S113069844800C4040800C4058800C4060800C40E2
S11306A878800C407C800C4020800C4080B500F0A1
S11306B808F82449096811F00F01C8402249086064
S11306C802BD2248006810F47050B0F5006F0BD0DA
S11306D8B0F5805F05D0B0F5005F08D11C4800680C
S11306E827E04FF4004024E01A48006821E01A4843
S11306F8006810F4E060002818D0B0F5807F13D0AB
S1130708B0F5007F0ED0B0F5407F09D0B0F5806F0A
S113071804D0B0F5A06F0BD110480AE0104808E0E7
S1130728104806E0104804E0104802E0104800E0D1
S11307380020704770474FF4004070470448006831
S11307487047000004800C40540700202C800C40A3
S113075804000020000000200C800C40003FAB0186
S1130768406F4001809FD500C0D8A700C0CF6A0061
S113077840420F00034800680149088070470000A0
S1130788600700202C800C40DFF800F09100002066
S1130798DFF800F00900002080B500F055FA5FF09A
S11307A8FF30DFF8941408605FF0FF30DFF88C1432
S11307B8086001BD70B504000D001600200000F0AB
S11307C8CFF9FF2805D02819401E00F0C9F9FF28E1
S11307D801D1002017E0600A4FF400714843DFF8A4
S11307E860140968884207D12B0032002100DFF821
S11307F84C0400F0EDF806E02B0032002100DFF88D
S1130808380400F0E5F870BD70B504000D00200050
S113081800F0A6F906002819401E00F0A1F9F6B266
S1130828FF2E02D0C0B2FF2801D1002005E001004C
S1130838C9B23000C0B200F04CF970BD80B50020D8
S11308480090DFF8F803006810F1010F01D10120CE
S113085837E00098DFF8E413496808180090009816
S1130868DFF8D8138968081800900098DFF8CC13CB
S1130878C968081800900098DFF8C01309690818B7
S113088800900098DFF8B41349690818009000989C
S1130898DFF8A8138969081800900098DFF89C13FA
S11308A8C969081800900098C04300900098401C3B
S11308B800906A460421DFF888030068B830FFF71F
S11308C879FF02BD0020DFF8781309680968081861
S11308D8DFF86C130968091D09680818DFF8601344
S11308E80968083109680818DFF8541309680C31D5
S11308F809680818DFF848130968103109680818E6
S1130908DFF83C130968143109680818CC490968E8
S1130918183109680818CA490968B83109680818F3
S1130928002801D1012000E00020704780B5C348A9
S1130938006810F1010F06D0C04800F08CF80028B8
S113094801D100200EE0BC48006810F1010F06D068
S1130958B94800F080F8002801D1002002E000F036
S113096884F9012002BDB6480068704780B5CA05FD
S113097801D000200BE002688A4201D1012006E080
S113098801604FF40072001D00F0A4F9012002BDBB
S113099838B504000D00A948844208D1A64C2900A2
S11309A82000FFF7E3FF002810D100200FE0A4483F
S11309B80068854203D1A14CA1480568EFE72000EF
S11309C800F049F80028EAD1002000E0200032BDF8
S11309D82DE9F04104000F0015001E00780A4FF4B9
S11309E8007101FB00F8206810F1010F07D141469E
S11309F82000FFF7BBFF002801D1002029E0206870
S1130A08404508D041462000FFF7C2FF0400002CEF
S1130A1801D100201DE02068381A2044071D00F089
S1130A286BF9201D381AB0F5007F0AD318F5007148
S1130A382000FFF7ADFF0400002C01D1002008E0DE
S1130A48271D287838707F1C6D1C761E002EE6D171
S1130A580120BDE8F081F8B505000124286800F0FC
S1130A687FF8C0B2FF2801D100201DE0002600E075
S1130A78761C802E16D2286810EB860705EB8600B4
S1130A884068009000F038F9042269463800FFF7FE
S1130A987BFE002801D0002404E0386800998842CD
S1130AA8E6D000242000C0B2F2BD66480078C0B287
S1130AB8472802D0C0B2492802D14FF4007007E099
S1130AC8C0B2482802D14FF4805001E04FF40060CE
S1130AD87047F8B505000C0020002900C0B2C9B25F
S1130AE8884201D200203AE028005549097AC0B268
S1130AF8884206D3524890F8B0002100C9B288420F
S1130B0801D200202BE0FFF7D0FF06002800C0B276
S1130B1800F052F805002000C0B200F04DF80700BC
S1130B282000C0B200F067F8C019401E401B401CEA
S1130B38B0FBF6F4002700E07F1C3800210080B2E7
S1130B4889B288420AD200F0D7F8BFB206FB075030
S1130B58FFF71EFE0028EFD0002000E00120F2BDC0
S1130B6838B50400002500E06D1CEDB20F2D21D22C
S1130B7800F0C2F83248EDB20C2101FB05F14058EF
S1130B888442F1D32E48EDB20C2101FB05F1405803
S1130B982B49EDB20C2202FB05F2114449680818EE
S1130BA88442E1D22648EDB20C2101FB05F1084448
S1130BB8007A00E0FF2032BD38B50500002400E0CB
S1130BC8641CE4B20F2C13D200F096F81C48E4B26B
S1130BD80C2101FB04F10844007A2900C9B28842B7
S1130BE8EED11748E4B20C2101FB04F1405801E0AE
S1130BF85FF0FF3032BD38B50500002400E0641C06
S1130C08E4B20F2C14D200F077F80D48E4B20C21AA
S1130C1801FB04F10844007A2900C9B28842EED1E4
S1130C280748E4B20C2101FB04F10844406800E0E1
S1130C38002032BD00000000780200207C0400205F
S1130C48DC190000FE81E00F1048006850F0010034
S1130C580E49086041F671300D4908600B48006878
S1130C68400840000949086070470848006850F087
S1130C780100064908600020054908600348006827
S1130C8840084000014908607047000008000C4013
S1130C983C000C4080B500F030F801BD10B500F000
S1130CA83CF8002810D000F061F800F0AEF800F02D
S1130CB838F8064908400649086000F032F8001D73
S1130CC8046800F01CF8A04710BD000080FFFF1F57
S1130CD808ED00E070B504000D00160005E0287862
S1130CE820706D1C641C00F007F83000461E80B2AA
S1130CF80028F4D170BD7047704772B6704762B669
S1130D08704780B5FFF748FD01BD80B5FFF752FD78
S1130D1802BD80B5FFF778FD02BD80B5FFF7D2FDAF
S1130D2802BD80B5FFF71FFE02BD80B5FFF786FD43
S1130D38002801D1002001E0FFF7F8FD02BD000002
S1130D4880B500F07FF800F0C1FA0020224908704D
S1130D5801BD80B5214800F027FB012805D10020FA
S1130D681D4908701D4800F097F801BD704780B50B
S1130D78194A1278002A02D1C9B200F0E8FA00F040
S1130D8885F801BD14480078002805D0022807D04A
S1130D9804D3032806D007E0402006E0002004E03E
S1130DA8002002E0002000E0402080B270470A489A
S1130DB80078002805D0022807D004D3032806D0D9
S1130DC807E0402006E0002004E0002002E00020C4
S1130DD800E0402080B27047740100201007002012
S1130DE880B500F04AF802BD80B500F00EF843F271
S1130DF8AF601049086000200F49086005200F49BA
S1130E08086000200E49086001BD00200B490860F5
S1130E1870470A480068C00304D509480068401CA4
S1130E2807490860704780B5FFF7F3FF0448006876
S1130E3802BD000014E000E018E000E010E000E06B
S1130E48580700200020DFF8601408700020DFF83D
S1130E58581488640020DFF8501481F843000020F7
S1130E68DFF84414A1F844000020DFF83C1488702B
S1130E780020DFF8341448707047DFF82C04007839
S1130E88002801D1002000E0012070470020DFF88D
S1130E98181481F84300704780B50178FF291ED1E2
S1130EA800F091F8DFF8000490F84300012802D11B
S1130EB8102000F07EF8DFF8F003B0F944000128B0
S1130EC80CDB0120DFF8E01381F84300DFF8D803D6
S1130ED8B0F94410DFF8D40300F053F801BDDFF88B
S1130EE8C813097801294BD10178C92932D0CC29F2
S1130EF83FD0CF293AD0D0292FD0D12933D0D229E5
S1130F082ED0F32917D0F4290FD0F5290AD0F629C1
S1130F180ED0FA2912D0FC2913D0FD2914D0FE29A9
S1130F2815D029E000F0D1F8BCE700F0F1F8B9E7F2
S1130F3800F0C0F8B6E700F011F9B3E700F0A2F842
S1130F48B0E700F09AF8ADE700F07FF8AAE700F000
S1130F586EF8A7E700F035F9A4E700F054F9A1E723
S1130F6800F013F99EE700F080F99BE700F091F98F
S1130F7898E700F0A3F995E7202000F01AF891E724
S1130F88ACE780B589B2FFF7F2FE01BD10B40023C7
S1130F9802E00478E318401C0C00611E002CF8D110
S1130FA8DBB21360012010BC70470020BE494870B2
S1130FB87047FE21BC4AD170BB4908710220BA4966
S1130FC8A1F84400704780B5FFF7EFFF0120B64948
S1130FD80870FF20B449C8700020B3490871B248AA
S1130FE8007950F01000B04908710020AE494871EA
S1130FF8AD484079AC494871FFF7C4FEAA498871E5
S1131008FFF7D5FEA849C871FFF7D1FE80B2000AE0
S1131018A54908720120A44948720120A24988728E
S11310280820A149A1F84400FFF76BFE01BD80B573
S113103800209D490870FFF7B8FFFF209A49C8703F
S113104801209949A1F8440001BDFF209649C870C0
S113105800209549087194484078934948710020C4
S11310689149887100209049C87100208E490872FE
S113107806208D49A1F84400704780B50020FFF789
S113108898FF01BDFF208849C8708948864988644B
S1131098002085490871002083494871002082494D
S11310A8887107208049C1F8070008207E49A1F803
S11310B844007047FF217C4AD17040687A498864AB
S11310C801207949A1F84400704710B50400FFF7DE
S11310D859FE80B2401E6178884203DA2220FFF765
S11310E868FF14E0627892B26F48816C7148FFF728
S11310F8F1FDFF206C49C8706B48806C6178081852
S1131108694988646078401C6749A1F8440010BDA7
S113111810B50400FFF736FE80B2401E617888429D
S113112803DA2220FFF745FF17E060685E49886408
S1131138627892B25C48816C5E48FFF7CBFDFF2071
S11311485949C8705848806C6178081856498864A9
S11311586078401C5449A1F8440010BD80B5FF21B3
S1131168514AD170544A41684F48806CFFF70EFFCA
S11311784D49087100204C49487100204A4988713A
S113118808204949A1F8440001BD80B5FF2046491B
S1131198C870002044490871002043494871FFF78A
S11311A8F1FD4149887100203F49C87100203E493A
S11311B8087200203C49487207203B49A1F84400C2
S11311C801BD10B50400FFF7DDFD621C80B2411EAD
S11311D83548806CFFF799FD002803D13120FFF7CB
S11311E8E8FE0FE0FF203049C870FFF7CBFD2E4919
S11311F8896C80B2401E40182B49886401202A4912
S1131208A1F8440010BD10B50400FFF7BBFD80B27F
S1131218801E6178884203DA2220FFF7CAFE23E0A1
S1131228FF202149C87001201F49A1F844006078B3
S1131238002807D1FFF779FD002802D13120FFF7F4
S1131248B8FE11E0A21C61781748806CFFF75DFDB9
S1131258002803D13120FFF7ACFE05E01248806C6A
S1131268617808181049886410BD80B541680E4833
S1131278806CFFF74EFD002803D13120FFF799FE5B
S113128806E0FF200849C87001200749A1F8440076
S113129801BD80B5FFF702FDFF200349C870012096
S11312A80149A1F8440001BD8006002083060020FE
S11312B8AC1C0000840600208706002080B531207D
S11312C8FFF777FE01BD00004163704700B585B0A4
S11312D868466A49102200F0EFF801216848FFF7D0
S11312E815F8012304220621022000F021F9002325
S11312F801220721022000F01BF901216148FFF7B0
S113130805F802216048FFF705F901215F48FEF757
S11313185AFF01215D48FEF7F9FF00208DF800000F
S113132869465B4800F0BDF94FF41652002158484D
S113133800F075F903205749086004215448FFF761
S1131348C3FF0521524800F091F905B000BD70B5FE
S113135804000D00EDB2412D03DB6C214E4800F072
S1131368D6F92800C0B200F073F8C0B2012803D03F
S11313787021494800F0CBF900260DE0FFF7BCFCCA
S1131388B6B2A05D00F064F8C0B2012803D0792198
S1131398414800F0BCF9761C30002900C9B280B27B
S11313A889B28842EAD370BD10B504003B4800787E
S11313B8002813D13A4800F03DF8012838D13848BC
S11313C80078002834D0FFF72EFD36490860002045
S11313D83549087001203149087029E030483249FC
S11313E809780844401C00F025F8012816D12E4835
S11313F80078401C2C4908702B4800782849097843
S1131408884215D12848027892B228492000FFF76B
S113141861FC00202149087001200AE0FFF703FD60
S1131428204909686431814202D200201B490870AE
S1131438002010BD10B5040000201D4909684907A3
S113144804D5134800F050F920700120C0B210BD33
S113145880B518490968C90601D400200CE00100C8
S1131468C9B20B4800F046F901E0FFF745FC114802
S11314780068C006F9D5012002BD0000801C0000E8
S113148800C20200002304000300120040151600E5
S11314980044084054440840A41B0000640700208A
S11314A8CC0600205C07002063070020CD0600203E
S11314B82C44084008440840103A07D330B4B1E833
S11314C83810103AA0E83810F9D230BC530724BFBA
S11314D8B1E80810A0E8081044BF51F8043B40F8EC
S11314E8043BD20724BF31F8022B20F8022B44BF57
S11314F80B7803707047083A07D3B1E80810083A24
S113150840F8043B40F804CBF7D25307E4E7000063
S11315183E4AC0B2242303FB00F3D2589208920037
S1131528C9B21143394AC0B22423584311507047F1
S113153870B4D2B2002A14D0002B09D001248C40F4
S1131548324DC0B2242606FB00F635442C6108E06F
S113155801248C402D4DC0B2242606FB00F63544E8
S11315686C6108291BD2294CC0B2242505FB00F55F
S11315782C4464680F250E00F6B2B600B540AC439F
S1131588D2B20D00EDB2AD0012FA05F52C431F4D91
S1131598C0B2242606FB00F635446C601CE01B4CE4
S11315A8C0B2242505FB00F52C44A4680F250E00C1
S11315B8083EF6B2B600B540AC43D2B20D00083DC1
S11315C8EDB2AD0012FA05F52C43104DC0B2242635
S11315D806FB00F63544AC60D2B2002A14D1002BC5
S11315E809D0012212FA01F1084AC0B2242358434F
S11315F81044016108E0012212FA01F1034AC0B261
S1131608242358431044416170BC70470060004073
S1131618026CD20702D4426C0A42FCD1704738B536
S113162804001500002906D10C4884420ED10C4848
S1131638FEF7A0FE01004801B0FBF5F5203DED00E2
S113164804212000FFF7E4FFE56031BD054884422A
S113165801D10548ECE7F8E7000000000040084025
S113166840051400004408404015160038B504002D
S1131678C9B2CD4315F005056D00C9B20D43022169
S11316882000FFF7C5FF656031BDC9B2002905D048
S1131698416C0029FCD10121016401E000210164AD
S11316A8704738B504000D0002212000FFF7B0FF91
S11316B80A20606001212000FFF7E7FF206830F06E
S11316C81C00297B0843697B0843A97B08432060E5
S11316D8AA6869682000FFF7A2FF287860600021E3
S11316E82000FFF7D2FF31BD81688906FCD5C069A7
S11316F8C0B2704738B504000D00A068C006FCD518
S113170840212000FFF784FFEDB2A56231BD80B50A
S1131718FFF7F2FAFCE7000080B568480168080E94
S113172800280DD16648026832F0700202606548EC
S1131738026822F060420260026872F0606202602D
S1131748080E042813D25F48016831F4FC51016083
S11317585D48002101605D48002101605C4800216A
S113176801605C48002101605B4800210160684613
S113177800F0DCF89DF80000012811D19DF8010063
S1131788002804D15048016851F0020101609DF815
S11317980100022804DA4D48016851F00101016092
S11317A84E4801684E48814224D24848016851F4A1
S11317B8904101604B480068000410F0FE4149481C
S11317C80068000410F4FE0001434648006810F461
S11317D8FE4001434348006810F07F00014342483B
S11317E8016042484249096801603848016831F497
S11317F89041016001BD80B500F005F800F0ACF837
S113180800F0B8F8FCE780B5FEF794FFFFF784FF13
S1131818012201210020FEF7E1FE2B48006850F068
S11318280F00294908602948006840F47F4050F0B7
S1131838FF002649086000212E48FEF767FD0021B5
S11318482D48FEF763FD00212C48FEF75FFD0021BB
S11318582B48FEF75BFD00212A48FEF757FD0021BF
S11318682948FEF753FD00212848FEF74FFD0021C3
S11318782748FEF74BFD00212648FEF747FD0021C7
S11318882548FEF743FD00212448FEF73FFD0021CB
S11318982348FEF73BFD00212248FEF737FD0021CF
S11318A82148FEF733FD0123052209210120FFF712
S11318B83FFE02210120FFF72BFE01BDFC81E00F52
S11318C80CA00C4020600C4040800C4044800C402C
S11318D858800C4060800C4078800C40F081E00F08
S11318E800BA8A4CB481E00F342000402C400040F8
S11318F8C881E00F0003040000130400003304004F
S113190800A20200000202000012020000220200EB
S113191800320200007202000082020000B20200DB
S113192800E2020000F2020000D20200074909683E
S113193811F03F0101700649096811F0F001054AE8
S11319481268C2F30312114341707047E0FF0FE0BD
S1131958E8FF0FE0ECFF0FE080B5FFF79BF9FFF716
S1131968CAF9FFF741FAFFF7CCF9FFF7E9F900F0F4
S11319780BF801BD80B5FFF7BFF9FFF74AFAFFF787
S1131988E8F900F00CF801BD80B501200F49087092
S1131998FFF749FA0E49086000F001F801BD80B567
S11319A8FFF71EFA012810D00848007801280CD146
S11319B8FFF739FA0649096811F5FA71884204D320
S11319C8002002490870FFF769F901BD6207002089
S11319D85007002000200000002000000100000043
S11319E80040000000200000020000000060000029
S11319F80020000003000000008000000020000018
S1131A080400000000A00000002000000500000001
S1131A1800C00000002000000600000000E00000F4
S1131A280020000007000000000001000020000062
S1131A380800000000200100002000000900000048
S1131A4800400100002000000A00000000600100BE
S1131A58002000000B0000000080010000200000AE
S1131A680C00000000A00100002000000D00000090
S1131A7800C00100002000000E00000000E001008A
S1131A88002000000F000000F0B401684468836877
S1131A98014401EB5402E40748BF4B44914202D18C
S1131AA8F0BC0C30704711F8015B15F0030604BF55
S1131AB811F8014BE61C2C090F2C07D111F8014B26
S1131AC80F3403E011F8017B03F8017B761EF9D18A
S1131AD8002CE3D0AD0811F8016B05F00305032DC4
S1131AE808BF11F8015B06EB05256D42A41C1D44D3
S1131AF8D4D015F8016B03F8016B641EF9D1CDE756
S1131B08433A5C576F726B5C736F66747761726586
S1131B185C4F70656E424C545C5461726765745CCA
S1131B2844656D6F5C41524D434D335F45464D33BB
S1131B38325F4F6C696D65785F454D33324738388D
S1131B48304631323853544B5F4941525C426F6FCF
S1131B58745C766563746F72732E630019E050F8D1
S1131B68041BCB0744BFA9F101035918121F002312
S1131B78042A41F8043BF9D25FEA827C0B4604D577
S1131B884FF0000CA1F800C09B1CD10744BF0021F2
S1131B98197050F8042B002AE1D17047433A5C5776
S1131BA86F726B5C736F6674776172655C4F706596
S1131BB86E424C545C5461726765745C536F757201
S1131BC863655C41524D434D335F45464D33325C4A
S1131BD8756172742E63000010B507497944183191
S1131BE8064C7C44163404E00A68081D11448847EE
S1131BF80146A142F8D110BD0800000024000000ED
S1131C085DFFFFFFF00400007802002000000000E0
S1131C1879FEFFFF980000004A020000000000203F
S1131C2800F00BF8002801D0FFF7D6FF0020AFF32F
S1131C380080FFF7E0FD00F002F80120704700F093
S1131C4801B800000746384600F002F8FBE7000038
S1131C5880B5AFF30080024A11001820ABBEFBE741
S1131C6826000200034B9D46AFF30080AFF30080CB
S1131C78FFF7D6FF780200200500000000000000EE
S1131C88802500000000000080B53C210148FFF7D2
S1131C983EFD01BD081B0000AFF30080AFF30080D8
S1131CA8FFF7BEFF4F70656E424C5400101B00488E
S1131CB8E801008000005449554A126852F00102B4
S1131CC8534B1A60534A10600120520620075248A9
S1131CD80068400708D54D08100C0840004B490817
S1131CE8605FF0FF3029E04C1212801A52471A1232
S1131CF8451A10077FF001001CE00220443A100343
S1131D0800E0491E431C500BC00701D50029F8D137
S1131D18002908D13C2C323A2C5003020006E03743
S1131D281212351210270020704730B4334B1B6849
S1131D3853F00103314C23609310002200E0521C3D
S1131D489A424FDA00EB82042D4D2C6001242C06B4
S1131D5810032C4C2468647E5227405225981001A5
S1131D6842E0261A12A41A52211A521F981010354A
S1131D78E01B4C00E0641E1E4D2D682D0701D400A5
S1131D882C9450022C08D11728521594100521E0E0
S1131D9851F822401564100108241206320E361236
S1131DA8103622EDCA31365001B5D109367207CA48
S1131DB85205123203CA100B30BC70478096980043
S1131DC808000C401004120C04121C04121804021B
S1041DD80402
S9031CA13F
